:0200000480007A
:100000006F000005732F2034930F80006308FF03F7
:10001000930F90006304FF03930FB0006300FF038E
:10002000130F000063040F0067000F00732F2034CC
:1000300063540F006F00400093E19153171F0000BD
:1000400023223FFC171F000023200FFC6FF01FFF2F
:100050009300000013010000930100001302000050
:100060009302000013030000930300001304000038
:100070009304000013050000930500001306000020
:100080009306000013070000930700001308000008
:10009000930800001309000093090000130A0000F0
:1000A000930A0000130B0000930B0000130C0000D8
:1000B000930C0000130D0000930D0000130E0000C0
:1000C000930E0000130F0000930F0000732540F102
:1000D0006310050097020000938202017390523072
:1000E000735044749702000093820201739052305F
:1000F00073500018970200009382420273905230AE
:100100009B021000939252039382F2FF7390023B82
:100110009302F0017390023A73504030970200004E
:1001200093824201739052307350203073503030BC
:100130009301000097020000938202ED7390523009
:10014000130510001315F501635C05000F00F00F97
:10015000930110009308D005130500007300000000
:1001600093020000638A020073905210B7B200003D
:100170009B829210739022307350003097020000DF
:100180009382420173901234732540F17300203042
:10019000930120009B00F0FF9390700213D7004062
:1001A0009B03F0FF939373026314772A930130004B
:1001B000B700008013D71040B70300C0631A772838
:1001C00093014000B700008013D77040B70300FFD1
:1001D0006310772893015000B700008013D7E040E8
:1001E000B703FEFF6316772693016000B700008017
:1001F0009B80100013D7F0419303F0FF631A77241C
:1002000093017000B70000809B80F0FF13D700407F
:10021000B70300809B83F3FF631C77229301800068
:10022000B70000809B80F0FF13D71040B703004059
:100230009B83F3FF631E772093019000B70000803B
:100240009B80F0FF13D77040B70300019B83F3FF3F
:10025000631077209301A000B70000809B80F0FF1F
:1002600013D7E040B70302009B83F3FF6312771EAE
:100270009301B000B70000809B80F0FF13D7F041DE
:10028000930300006316771C9301C000B78081813F
:100290009B80101813D70040B78381819B8313186C
:1002A0006318771A9301D000B78081819B80101862
:1002B00013D71040B7C3C0C09B83030C631A7718D1
:1002C0009301E000B78081819B80101813D77040A4
:1002D000B70303FF9B833330631C77169301F00051
:1002E000B78081819B80101813D7E040B703FEFFD1
:1002F0009B836360631E771493010001B780818143
:100300009B80101813D7F0419303F0FF631277140A
:1003100093011001B700008093D07040B70300FF35
:10032000639870129301200113020000B70000804F
:1003300013D770401303070013021200930220002A
:10034000E31652FEB70300FF6314731093013001EC
:1003500013020000B700008013D7E0401300000034
:10036000130307001302120093022000E31452FE4D
:10037000B703FEFF631E730C9301400113020000DC
:10038000B70000809B80100013D7F04113000000DD
:100390001300000013030700130212009302200051
:1003A000E31052FE9303F0FF6314730A93015001AC
:1003B00013020000B700008013D770401302120030
:1003C00093022000E31852FEB70300FF6312770880
:1003D0009301600113020000B700008013000000C9
:1003E00013D7E0401302120093022000E31652FEDE
:1003F000B703FEFF631E7704930170011302000030
:10040000B70000809B801000130000001300000064
:1004100013D7F0411302120093022000E31252FEA0
:100420009303F0FF631677029301800193504040DD
:1004300093030000639E70009301900193001002EB
:1004400013D0A040930300006314700063103002C7
:100450000F00F00F638001009391110093E11100F0
:100460009308D00513850100730000000F00F00F02
:10047000930110009308D0051305000073000000DD
:10048000731000C000000000000000000000000029
:10049000000000000000000000000000000000005C
:1004A000000000000000000000000000000000004C
:0C04B00000000000000000000000000040
:1010000000000000000000000000000000000000E0
:1010100000000000000000000000000000000000D0
:1010200000000000000000000000000000000000C0
:1010300000000000000000000000000000000000B0
:081040000000000000000000A8
:040000058000000077
:00000001FF
